:10000000F9C0000013C1000011C100000FC10000C1
:100010000DC100000BC1000009C1000007C10000B4
:1000200005C1000003C1000001C100000C941012C2
:10003000FDC00000FBC00000F9C000008AC700003E
:10004000F5C00000F3C00000F1C0000093C1000043
:10005000EDC00000EBC00000E9C00000E7C00000F8
:10006000E5C00000E3C00000E1C00000DFC0000008
:10007000DDC0000012011001FF000010EB0304219D
:10008000000201020301040309040C0341005400AF
:100090004D0045004C00000018034100560052007E
:1000A00049005300500020006D006B0049004900DA
:1000B000000009000A000A000B000C000D000D00F2
:1000C0000E000F00100010001200130013001400A7
:1000D00016001600180019001A001C001D001F0051
:1000E0002000220023002500270029002B002E00DD
:1000F00030003200340037003A003D004000430039
:1001000046004A004E00520055005A005E0063004F
:1001100068006D00730078007E0084008B00910001
:100120009900A000A900B100B900C300CC00D6001E
:10013000E100EC00F700040111011E012D013B015B
:100140004B015B016C017D019101A501BA01CF0159
:10015000E601FE01160231024C026A028802A80280
:10016000CA02ED021103380360038B03B803E703EF
:1001700018044B048104B904F50434057505B90568
:1001800001064E069D06EF064807A307040865080A
:10019000D0084009B6092B0AAB0A300BC30B510C2F
:1001A000EE0C8F0D400EF60EAF0F681047111412B3
:1001B000F512ED13E214F015F9161B185C19911ADB
:1001C000E51B251D831E0320AB21302332250F277D
:1001D000F128F82A1A2D492FA1311434A1364539B6
:1001E000173C1A3F34426045DF48704C40004101E3
:1001F0004243030011241FBECFEFD2E0DEBFCDBFCC
:1002000011E0A0E0B1E0EAEEF7E202C005900D9245
:10021000A038B107D9F711E0A0E8B1E001C01D9204
:10022000A339B107E1F750D00C94F313E9CE85B1AF
:100230008F71806C85B9089585B18F71806485B99F
:10024000089556C008958EB3843089F4C9D182E0F0
:100250008093E9008091E80082FF09C085B18F7129
:10026000806C85B99CD085B18F71806885B90895FF
:1002700082E060E842E30E94691180FD02C090E4E0
:1002800001C090E885B18F71982B95B9089584B716
:10029000877F84BF88E10FB6F89480936000109246
:1002A00060000FBE80E090E020E80FB6F894209345
:1002B0006100809361000FBE84B1806E84B985B106
:1002C0008F7185B90C940112E2DF82D185B18F71F3
:1002D000806485B97894489902C090E201C090E0AA
:1002E00085B18F7D982B95B9AEDF0E94C513F3CFF2
:1002F000DA01F9011082923049F0933069F09130BF
:1003000089F5E4E7F0E022E130E030C09083E0E0FE
:10031000F1E020E230E02AC0813059F0813028F04D
:10032000823059F08330F1F40EC0E6E8F0E08491B9
:1003300007C0EAE8F0E0849103C0E8E9F0E08491C6
:10034000282F30E013C080912001282F30E082E375
:1003500090E090932F0180932E0182E08083E0E271
:10036000F1E004C0E0E0F0E020E030E0ED93FC9349
:10037000C901089578941F920F920FB60F9211241D
:100380008F938AB5882321F08AB581508ABD01C038
:1003900015BC8F910F900FBE0F901F901895FF9274
:1003A0000F931F931091F10084E68ABD85E085BD0F
:1003B000143109F4CBC0153110F51A3009F4ADC071
:1003C0001B3068F4143038F4123008F054C0113087
:1003D00009F0D4C033C0163009F0D0C078C0113154
:1003E00009F4AFC0123120F4103109F0C7C0A7C022
:1003F000123109F4AEC0133109F0C0C0A4C01931E4
:1004000009F4ACC01A3168F4163109F49FC01631F2
:1004100008F499C0173109F4A1C0183109F0AEC031
:100420009AC01D3109F49DC01D3108F494C01035E7
:1004300009F49BC0113509F0A1C095C08091E80076
:100440008B778093E80082E08093E9008091EC0054
:1004500081608093EC001093F1001092F1008AE02B
:100460008093F1008EE391E06AE070E040E050E0BC
:100470000E94171199C00091F100123011F0FF2471
:1004800002C0F090F1008091E8008B778093E80043
:1004900082E08093E9008091EC0081608093EC0021
:1004A0001093F100802FB5D0123041F481FF0DC0C0
:1004B0001092F100802F6F2DB4D076C080FF05C060
:1004C0001092F100802F9DD06DC080EC6BC084E84D
:1004D00091E064E070E040E050E00E947310809191
:1004E000E8008B778093E80082E08093E9008091B8
:1004F000EC0081608093EC008091840190918501F3
:10050000A0918601B0918701B7FF03C081E080937D
:10051000830186E08093F1000FC08091E8008B7723
:100520008093E80082E08093E9008091EC00816094
:100530008093EC001093F1001092F10035C06DD45F
:1005400038C037D436C0812F04D333C0812F53D263
:1005500030C002D22EC0812FF7D02BC0812FAED059
:1005600028C05DD126C034D624C06CD722C080916B
:10057000E8008B778093E8000E949C118091F20044
:100580008034A9F38091E8008B778093E80082E0C3
:100590008093E9008091EC0081608093EC001093DF
:1005A000F10089EC8093F1008091E8008E778093D0
:1005B000E80015BC0E949C1182E08093E9008091C4
:1005C000EC008E7F8093EC001F910F91FF900895B7
:1005D0008BE987BD82E084BD80936E003AD0E9C488
:1005E0000895982FE9E4F1E08081981741F081E0C7
:1005F000E436F80711F03396F7CFE0E0F0E0CF01F2
:100600000895EFDFFC01009711F480E008958281E6
:100610000895E7DFFC01009711F480E008958181DF
:1006200008950F931F93182F062FDBDFFC0100970F
:1006300069F002831E3919F480E090E004C0183993
:1006400029F481E090E0602F0E94E1131F910F9147
:1006500008950F931F9380E090E00E94D913182F04
:1006600081E090E00E94D913082F1F3F21F08EE90E
:10067000B8DFFC0112830F3F21F088E9B2DFFC01F3
:1006800002831F910F910895282F40EA5FE003C075
:10069000CA010197F1F7222321F08AB5215088235E
:1006A000B9F70895982F80916701882329F09EBD9E
:1006B0000DB407FEFDCF0895892FBBC4DF92EF92E2
:1006C000FF920F931F93DF93CF9300D000D0CDB74D
:1006D000DEB7D82E8E010F5F1F4FC80164E070E0B7
:1006E00040E050E00E94C5108091E8008B77809335
:1006F000E80082E08093E9008091EC0081608093C3
:10070000EC0085E0E82EF12CEC0EFD1EF801819145
:100710008F01C8DF0E151F05C9F7D092F1001092A6
:10072000F1001092F1008091E8008E778093E8004C
:100730000F900F900F900F90CF91DF911F910F911D
:10074000FF90EF90DF900895BF92CF92DF92EF92EB
:10075000FF920F931F93DF93CF93CDB7DEB7299707
:100760000FB6F894DEBF0FBECDBFB82ECE010596F2
:1007700065E070E040E050E00E94C5108091E80024
:100780008B778093E80082E08093E9008091EC0011
:1007900081608093EC008E010A5F1F4F7E010894F8
:1007A000E11CF11C9AE0C92ED12CCC0EDD1EF80103
:1007B000908180916701882331F09EBD0DB407FEC2
:1007C000FDCF8EB502C0892F34D4F70181937F010C
:1007D0000F5F1F4F0C151D0551F7B092F1001092DD
:1007E000F1008D81FE01E80FF11D80818093F10001
:1007F0001092F1008091E8008E778093E8002996AE
:100800000FB6F894DEBF0FBECDBFCF91DF911F9121
:100810000F91FF90EF90DF90CF90BF900895EF92EF
:10082000FF920F931F93DF93CF93CDB7DEB7C250E4
:10083000D1400FB6F894DEBF0FBECDBFCE010196FA
:1008400063E070E040E050E00E94C51034E0E32E29
:10085000F12CEC0EFD1E6981C70170E040E050E014
:100860000E94C5108091E8008B778093E80082E0B9
:100870008093E9008091EC0081608093EC008DE131
:100880008093F1001092F10000E00BC089810817FD
:1008900028F4F701E00FF11D808101C080E002DF44
:1008A0000F5F8B81081790F310E024E0E22EF12C0B
:1008B000EC0EFD1E2CC0898190916701081778F419
:1008C000F701E00FF11D8081992331F08EBD0DB449
:1008D00007FEFDCF8EB501C0ACD30F5F0AC09923D0
:1008E00031F01EBC0DB407FEFDCF8EB502C080E016
:1008F000A0D38093F1008091E80085FD07C080912E
:10090000E8008E778093E8000E949C111F5F8A8127
:10091000181788F21092F1009091E8008091E80099
:100920008E778093E80095FD09C00E949C1180910C
:10093000E8008E778093E8000E949C11CE5FDE4F26
:100940000FB6F894DEBF0FBECDBFCF91DF911F91E0
:100950000F91FF90EF900895EF92FF920F931F93E6
:10096000DF93CF9300D000D000D0CDB7DEB7CE015B
:10097000019666E070E040E050E00E94C510809172
:10098000E8008B778093E80082E08093E900809113
:10099000EC0081608093EC008E010D5F1F4F47E0FB
:1009A000E42EF12CEC0EFD1EF80181918F017ADE10
:1009B0000E151F05C9F78A81882321F4898164DE19
:1009C00090E002C061D3982F82E18093F100909370
:1009D000F1008091E8008E778093E80026960FB6AC
:1009E000F894DEBF0FBECDBFCF91DF911F910F9165
:1009F000FF90EF900895DF92EF92FF920F931F9375
:100A0000DF93CF9300D00F92CDB7DEB7F82ECE0193
:100A1000019663E070E040E050E00E94C5109981CB
:100A20008A8189839A838091E8008B778093E8009C
:100A300082E08093E9008091EC0081608093EC007B
:100A4000F092F1001092F10000E010E068E0D62E84
:100A5000EE24E39459C080918301882319F032D3A6
:100A6000109283018B811EDE80918401909185011B
:100A7000A0918601B0918701892F9A2FAB2FBB27B8
:100A800011DE809184010EDE80916701882331F0B0
:100A90001EBC0DB407FEFDCF8EB502C080E0C9D2EA
:100AA0008093F1008091E80085FD07C08091E80007
:100AB0008E778093E8000E949C1124E1F21619F4CD
:100AC0008B818D258B8300FD03C086E1F816D1F460
:100AD0008091840190918501A0918601B091870158
:100AE0000196A11DB11D8093840190938501A0936F
:100AF0008601B093870126E1F21621F0892B11F4CB
:100B0000E09283010F5F1F4F89819A8108171907AF
:100B100008F4A1CF1092F1009091E8008091E800D4
:100B20008E778093E80095FD09C00E949C1180910A
:100B3000E8008E778093E8000E949C110F900F9040
:100B40000F90CF91DF911F910F91FF90EF90DF9069
:100B500008954F925F926F927F928F929F92AF9281
:100B6000BF92CF92DF92EF92FF920F931F93DF938A
:100B7000CF93CDB7DEB7C950D1400FB6F894DEBFE2
:100B80000FBECDBF182FCE01019669E070E040E0A6
:100B900050E00E94C5106A81798181E06130780758
:100BA00098F08091E8008B778093E80082E0809352
:100BB000E9008091EC0081608093EC001093F100DB
:100BC00080EC8093F100D8C07A836983CE010A96C5
:100BD00040E050E00E94C51089819A810A968F7387
:100BE0009070892B39F48091E8008B778093E8002E
:100BF0000E949C118091E8008B778093E80082E04E
:100C00008093E9008091EC0081608093EC001331C7
:100C100011F4888401C089846090840170908501FA
:100C2000EE24FF24FAE0AF2EB12CAC0EBD1ECC2476
:100C3000DD24E8E04E2E552453946DC0F5019080DC
:100C40000B8180918301882319F03CD2109283019B
:100C50008D8128DD8091840190918501A09186018C
:100C6000B0918701892F9A2FAB2FBB271BDD809175
:100C7000840118DD892D16DD133119F48D81842549
:100C80008D83E114F10481F4981471F0C0FE05C065
:100C9000133119F48F81886002C08F81877F8F8321
:100CA000E0908401F090850100FD12C0E114F10490
:100CB00021F403FD02C0097F0260802FB701482D97
:100CC0002C810F8108D2282F882361F5EE24FF2480
:100CD000C0FC02C01531C9F4809184019091850156
:100CE000A0918601B09187010196A11DB11D80934D
:100CF000840190938501A0938601B09387011331FD
:100D000021F4892B11F4509283010894A11CB11C89
:100D10000894C11CD11C89819A81C816D90608F48F
:100D20008DCF20E08B8187FF23C08E81BBDC872D98
:100D3000B9DC862DB7DC80E0B5DC8B8185FF06C091
:100D4000E114F10419F48F7C80618B838B81B701EE
:100D5000482D2C810F81BFD1282F133149F4809168
:100D6000840190918501892B19F481E0809383019E
:100D70001093F1002093F1008091E8008E7780932A
:100D8000E800C75FDE4F0FB6F894DEBF0FBECDBFE1
:100D9000CF91DF911F910F91FF90EF90DF90CF9057
:100DA000BF90AF909F908F907F906F905F904F908B
:100DB00008950F931F93DF93CF9300D0CDB7DEB785
:100DC000CE01019662E070E040E050E00E94C51064
:100DD00008EE10E0F80180818B77808382E08093B9
:100DE000E900ECEEF0E080818160808389814CDC59
:100DF00080E0B8D1F2D08A8147DCE1EFF0E081E118
:100E000080831082F80180818E7780830F900F900D
:100E1000CF91DF911F910F9108958F929F92AF9282
:100E2000BF92CF92DF92EF92FF920F931F93DF93C7
:100E3000CF93CDB7DEB72F970FB6F894DEBF0FBEB6
:100E4000CDBFCE0105966BE070E040E050E00E941F
:100E5000C5108091E8008B778093E80082E0809352
:100E6000E9008091EC0081608093EC001092840195
:100E70001092850110928601109287018F8104DC07
:100E80007DD181E06FD18E81FFDBBCE08B2E912C78
:100E90008C0E9D1E5E010894A11CB11CA0E1CA2EFF
:100EA000D12CCC0EDD1E2AC08985EEDBF8019081A5
:100EB00080916701882331F09EBD0DB407FEFDCF00
:100EC0008EB502C0892FB5D0F70181937F010F5FE6
:100ED0001F4F0C151D0541F78B858823D1F0FE01AE
:100EE000E80FF11D90818A85981799F080E03AD13A
:100EF0008E81CADB81E036D18E81C6DB988599234D
:100F000051F08AB5882339F0915098878401750192
:100F1000CBCF90E001C090EC80E18093F100909302
:100F2000F1008091E8008E778093E8002F960FB64D
:100F3000F894DEBF0FBECDBFCF91DF911F910F910F
:100F4000FF90EF90DF90CF90BF90AF909F908F90E9
:100F500008951F920F920FB60F9211248F93199933
:100F600008C08091800187FF02C02A9A1BC02A987E
:100F700019C080918001880F809380018091810148
:100F800081508093810180918101882321F4109206
:100F9000810082E086BB1B9B05C08091800181603F
:100FA00080938001199A8F910F900FBE0F901F9020
:100FB00018953E9A10926F0010928500109284004E
:100FC00081E090E0909389008093880080E4809392
:100FD000800089E0809381000895809167018823D3
:100FE00049F084B1897F84B985B1867F85B91CBCFD
:100FF0001DBC089584B1897F84B985B1867F85B988
:10100000D8CF92E090936F001092850010928400E8
:10101000E82FF0E0EE0FFF1FEC55FF4F8591949104
:101020009093890080938800109280001092810034
:1010300008958093800188E08093810180918001F0
:1010400087FF02C02A9A01C02A9810928500109248
:1010500084008AE08093810080918101882319F0C7
:101060008AB58823C9F71092810080918001089584
:10107000982F80916701882329F09EBD0DB407FE4B
:10108000FDCF0895892FD5CF80EFF2DF80E0F0DF2C
:1010900080E0EEDF80916701882331F01EBC0DB443
:1010A00007FEFDCF8EB502C080E0C3DF80FF03C026
:1010B0008AB5882349F78AB5882311F481E8089511
:1010C00080E008958DE4D4DF80E0D2DF8091860156
:1010D000CFDF80E0CDCFEF92FF920F931F937B0184
:1010E000142F90E08E778830910581F18930910539
:1010F00034F48230910559F0049759F50BC08032D1
:10110000910541F08034910509F1409711F5822F46
:10111000BBDA1FC0802FACDF8F2DAADF8E2DA8DF9A
:1011200080916701882331F01EBC0DB407FEFDCF0E
:101130008EB502C080E07DDF811719F48AB588235F
:1011400049F78AB5882329F490E804C09DDF982FD9
:1011500001C090E084E68ABD892F1F910F91FF9016
:10116000EF900895882339F0249A8EE94ADA88238B
:1011700019F42C9A089524982C98089588E941DA56
:10118000E82F8730D8F481E080936701F0E0E451E4
:10119000FE4FE491E061209A289A84B1866084B978
:1011A00023982B9AE6FF03C08DB5816002C08DB5F0
:1011B0008E7F8DBD2098E064ECBD0895109267018C
:1011C00084B1866084B985B1896085B98E2F19CFC5
:1011D000DF93CF930F92CDB7DEB7CE01019661E0DA
:1011E00070E040E050E0D1D78091E8008B778093A9
:1011F000E80082E08093E9008091EC0081608093B8
:10120000EC0099819093820181E58093F100913007
:1012100011F480EC01C080E08093F1008091E8003F
:101220008E778093E8000F90CF91DF910895AF9271
:10123000BF92CF92DF92EF92FF920F931F93DF93B3
:10124000CF93CDB7DEB7C850D1400FB6F894DEBF0C
:101250000FBECDBFCE01019668E070E040E050E0E7
:1012600094D73B812C819D818E817F8168856F839E
:1012700078878B839C832D833E83CE01099640E043
:1012800050E083D78F81988509968F739070892B52
:1012900039F48091E8008B778093E8000E949C11DC
:1012A0008091E8008B778093E80082E08093E900EA
:1012B0008091EC0081608093EC0080918201882312
:1012C00079F589818330A9F0843028F4813069F080
:1012D0008230A9F40CC0853031F0853008F44CC060
:1012E000863069F40AC088E048C044E209C04CE294
:1012F00007C045E383E366E305C04AE101C04EE26F
:1013000083E266E2EB80FC800D811E81AF80B884B1
:101310002A8199E0C92ED12CCC0EDD1EEDD208C059
:101320004F8158858B819C81BE01675F7F4FF4D4CC
:10133000882311F090E001C093E080E58093F100F4
:1013400084E08093F1009093F1008091E8008E7723
:101350008093E800C85FDE4F0FB6F894DEBF0FBE83
:10136000CDBFCF91DF911F910F91FF90EF90DF9054
:10137000CF90BF90AF9008958CE44B815C816D81DC
:101380007E81298520D3D4CFDF93CF93CDB7DEB72D
:10139000C750D1400FB6F894DEBF0FBECDBFCE010F
:1013A000019667E070E040E050E0EFD69A81EB8173
:1013B0007C816D816A837B83EC839D833E812F8159
:1013C0002E833F838091E8008B778093E80082E052
:1013D0008093E9008091EC0081608093EC00809123
:1013E0008201AE01485F5F4F882319F48E2F0DD321
:1013F00004C0CB01BA01A901C7D4882311F493E03A
:1014000001C090E080E58093F10085E08093F100D9
:101410009093F100992339F46E817F81CE01089673
:1014200040E050E004D78091E8008E778093E80098
:10143000C95FDE4F0FB6F894DEBF0FBECDBFCF91B0
:10144000DF910895DF93CF93CDB7DEB729970FB61D
:10145000F894DEBF0FBECDBF9091F100943009F437
:10146000ADC0953048F49230A1F1933008F04DC0F2
:10147000913009F03DC10AC0963009F4A3C09630FE
:1014800008F49EC0973009F033C1DEC08091E800B7
:101490008B778093E80082E08093E9008091EC00F4
:1014A00081608093EC0080918201882311F4ADD398
:1014B00005C0823011F090E002C0A6D4982F80E5DC
:1014C0008093F10081E08093F10089278093F100FF
:1014D0000AC18091E8008B778093E8009093E9003F
:1014E0008091EC0081608093EC00809182018823E0
:1014F00011F480D301C07DD480E58093F10082E0B7
:101500008093F1001092F100EEC0CE01059665E0E7
:1015100070E040E050E039D6588549857E816F8182
:101520004E835F83688779878091E8008B7780930B
:10153000E80082E08093E9008091EC008160809374
:10154000EC00809182019D81882339F59430C1F0AF
:10155000953038F4923071F0933080F49130D1F4BA
:101560000BC0963089F0963068F0973079F098305B
:1015700089F40EC080E20FC080E40DC088E60BC085
:1015800080E309C082E207C08AE205C082E303C0AB
:1015900088E101C080E089D207C0913011F084E178
:1015A00001C080E1BA019DD3882311F090E001C011
:1015B00093E080E58093F10083E091C038DE98C02D
:1015C000E3DE96C0CE01059661E070E040E050E0B9
:1015D000DCD58091E8008B778093E80082E08093EF
:1015E000E9008091EC0081608093EC0080918201A1
:1015F000882311F091E013C08D81813021F0823079
:1016000021F489E303C088E301C088E7BE016F5F6E
:101610007F4FB8D2882311F493E001C090E080E5B9
:101620008093F10086E08093F1009093F10099237C
:1016300009F059C089819A81AB81BC819D01442701
:1016400055272093F1004BC08091F100833039F190
:10165000843028F4813049F0823029F417C0843076
:1016600019F1853031F191E029C03091F1002091DC
:10167000F1009091F1008091F100809368019093C6
:10168000690120936A0130936B0117C09091F100BA
:101690008091F10080936C0190936D010EC0809158
:1016A000F10080936E0109C08091F10080936F0179
:1016B00004C08091F1008091F10090E08091E800F9
:1016C0008B778093E80082E08093E9008091EC00C2
:1016D00081608093EC0080E58093F10087E0809347
:1016E000F1009093F1008091E8008E778093E800FC
:1016F00029960FB6F894DEBF0FBECDBFCF91DF9114
:1017000008954D99FECF4D9BFECF4D99FECF5B9A2C
:10171000539A8091C9008F7E8093C9008091C9003F
:1017200088608093C90081E080938801089580914A
:101730008801882309F4E5DF80E04D99FECF4D9BB9
:10174000FECF4D99FECF8F5F8C30B9F70895109280
:101750008801249A2C9880E991E00197F1F78AB1E9
:1017600088628AB9529883E090E09093CD0080938C
:10177000CC0088E08093C9008FE68093CA00D7DF51
:10178000D6CF109288018AB188628AB952985B9A42
:1017900080E991E00197F1F783E090E09093CD002C
:1017A0008093CC0088E08093C9008FE68093CA00C4
:1017B000BEDFBDCF1F93182F80918801882309F4C5
:1017C000A0DF8091C80085FFFCCF8091C8008064B5
:1017D0008093C8001093CE001F9108958091C80097
:1017E00086FFFCCF8091C80080648093C800809100
:1017F000C900877F8093C9008091C9008061809370
:10180000C90053985B9810928801089580918801CF
:10181000882309F0E3DF8091C80087FD03C08AB503
:101820008823C9F78091CE0008958091880188238C
:1018300009F0D4DF8091C800806C8093C8001092BA
:10184000C9001092CA008AB1877D8AB98BB1837DA5
:101850008BB924982C98089580918801882309F0E9
:10186000BDDF80EC8093C8001092C9001092CA00BE
:101870008AB1877D8AB98BB1837D8BB90895EF9248
:10188000FF920F931F937B018C01862F93DFBB2761
:10189000A12F902F8F2D8EDFC801AA27BB278ADFAB
:1018A000E12EFF24002711278E2D84DF1F910F9139
:1018B000FF90EF90089590E0A0E0B0E020916801E3
:1018C0003091690140916A0150916B01822B932BF9
:1018D000A42BB52BBC01CD01D2CF8BE66BDF8FE003
:1018E000EADF80E267DF92DF982F8AB5882319F05C
:1018F00097FDF7CF81E008957F928F929F92AF92EC
:10190000BF92CF92DF92EF92FF920F931F93CF93EC
:10191000DF93882E962E742EE601D22E20FF10C063
:10192000DCDF882309F440C08CE444DF8AE0C3DFB5
:10193000892D40DF8CE43EDF8BE0BDDF81E03ADFC4
:10194000A114B104E9F0C9DF882371F18CE432DF1E
:101950008AE0B1DF882D2EDF8BE62CDFC801B701CE
:101960008EDF80EA27DF8A2D815024DF84E622DFA4
:10197000899120DF0894A108B108A114B104C1F72E
:10198000D1FE10C0AADF882379F08CE413DF8AE04F
:1019900092DF872D0FDF8CE40DDFC801B7016FDF09
:1019A00080E008DF81E001C080E0DF91CF911F91EE
:1019B0000F91FF90EF90DF90CF90BF90AF909F90EE
:1019C0008F907F900895CF92DF92EF92FF920F93C6
:1019D0001F93D82E7A018B01C22E7FDF882371F0EE
:1019E0008CE4E8DE8AE067DF8D2DE4DE8CE4E2DE65
:1019F000C801B70144DF8C2DDDDE81E01F910F911E
:101A0000FF90EF90DF90CF900895CF92DF92EF920A
:101A1000FF920F931F93CF93DF937B018C016A0199
:101A2000E9015BDF882369F18CE4C4DE8AE043DFEF
:101A300083E4C0DEC230D105C8F08BE6BBDEC8014E
:101A4000B7011DDF80EAB6DE9E012150822FB2DE93
:101A500084E2B0DE06C0DADEF60181936F012097E2
:101A600069F08AB521978823B1F708C08CE0A2DE1F
:101A7000C801B70104DFCADEF60180838AB581118F
:101A800081E0DF91CF911F910F91FF90EF90DF9058
:101A9000CF90089580E88EDEB9DE982F8AB588232E
:101AA00019F091FFF7CF81E00895CF92DF92EF9286
:101AB000FF921F93182F6A017B010FDF882309F41F
:101AC0005AC0103431F48CE475DE8AE0F4DE80E430
:101AD00039C0103309F03DC08CE46CDE8AE0EBDEE7
:101AE00086E368DE8CE466DE8BE0E5DE81E062DEC4
:101AF000F4DE882309F43FC08CE45CDE8AE0DBDEA0
:101B000083E358DE8BE656DEC701B601B8DE80EA15
:101B100051DE80916C0181504DDE84E64BDE10E099
:101B200003C080E047DE1F5F212F30E080916C0111
:101B300090916D0128173907A0F38CE43BDE8AE011
:101B4000BADE80E337DE8CE435DE8BE0B4DE81E0A4
:101B50000CC08CE42FDE8AE0AEDE812F2BDE8CE41D
:101B600029DEC701B6018BDE80E024DE93DF882307
:101B700019F081E001C080E01F91FF90EF90DF90AD
:101B8000CF9008951F93CF93DF93182FEB01188206
:101B900019821A821B82A1DE882339F18CE40ADEC5
:101BA0008AE089DE812F06DE8CE404DE8BE083DEB2
:101BB00081E000DE6FDF8823C1F08FDE8823A9F08B
:101BC0008BE6F8DD84E077DE80EAF4DD82E0F2DDAA
:101BD00084E2F0DD1BDE888319DE898317DE8A83C9
:101BE0008AB5882319F081E001C080E0DF91CF91B0
:101BF0001F9108954FDF81ECDDDD80E0DBDD81E8C2
:101C0000D9DD04DE8823B9F727CEEF92FF920F9338
:101C10001F93DF93CF93CDB7DEB728970FB6F89415
:101C2000DEBF0FBECDBFADDD81ECC4DD89E5C2DD19
:101C300082ECC0DD82E0BEDD80EEBCDD8E01085F9F
:101C40001F4F7E010894E11CF11CD701E0E7F1E091
:101C500088E001900D928150E1F7F8018081AADDC2
:101C6000015010400C171D0781F714DF28960FB69E
:101C7000F894DEBF0FBECDBFCF91DF911F910F91C2
:101C8000FF90EF900895282F8F70806930E02073C7
:101C90003070220F331F822B8DCD0F931F93182F7F
:101CA000092F88E687DD812F85DD89E683DD802F9A
:101CB00081DD1F910F91089520916F01822F8F7008
:101CC000806130E020733070220F331F822B72DD71
:101CD0009DDD982F8AB5882319F097FDEDCF81E01F
:101CE00008951F93CF93DF93182FEB01E5DF88232F
:101CF00079F080916E01C7DF812F5CDDCE018160BC
:101D0000CCDF80E657DD80E055DDD6DF811181E054
:101D1000DF91CF911F910895EF92FF920F931F9340
:101D2000CF93DF937C018B01EA01C6DF882321F189
:101D3000C0FF06C0F801EC0FFD1F8FEF80832196D6
:101D400080916E01A0DF8DE135DDC701A6DF10C0F7
:101D5000B3DF882389F084E62DDDF80180812ADD58
:101D600084E628DDF80181810E5F1F4F23DD229775
:101D7000209771F781E001C080E0DF91CF911F9142
:101D80000F91FF90EF900895EF92FF920F931F93A2
:101D9000CF93DF938C017B01EA018EDF8823B9F0BA
:101DA00080916E0170DF80E005DDC80176DF06C03E
:101DB00084E200DD2BDDF70181937F01209721F084
:101DC0008AB521978823A1F78AB5811181E0DF9137
:101DD000CF911F910F91FF90EF90089580E8EADC7A
:101DE00015DD982F8AB5882319F091FFF7CF81E090
:101DF0000895F4DF80ECDEDC80E0DCDC80E8DADC17
:101E000005DD8823B9F711CDEF92FF920F931F9351
:101E1000DF93CF93CDB7DEB728970FB6F894DEBF28
:101E20000FBECDBF94DC82ECC5DC82E0C3DC80EE6B
:101E3000C1DC8E01085F1F4F7E010894E11CF11C7C
:101E4000D701E8E7F1E088E001900D928150E1F7D9
:101E5000F8018081AFDC015010400C171D0781F79D
:101E6000BDDF28960FB6F894DEBF0FBECDBFCF9171
:101E7000DF911F910F91FF90EF9008959C01409189
:101E80009101509192014617570718F4F90190E01B
:101E90003CC06115710511F0AB01F8CF8091E800ED
:101EA0008E778093E80040E050E0F0CF8EB3882337
:101EB00009F440C0853009F43FC08091E80083FDFB
:101EC0003DC08091E80082FD2FC08091E80080FF36
:101ED0001CC08091F200282F30E007C081918093D0
:101EE000F100415050402F5F3F4F4115510519F00F
:101EF0002031310598F390E02031310509F491E06B
:101F00008091E8008E778093E8004115510571F6C5
:101F1000992361F609C08EB3882361F0853061F0A2
:101F20008091E80083FD0AC08091E80082FFF3CF32
:101F300080E0089582E0089583E0089581E00895A7
:101F40009C0140919101509192014617570718F456
:101F5000F90190E03DC06115710511F0AB01F8CFBA
:101F60008091E8008E778093E80040E050E0F0CF69
:101F70008EB3882309F441C0853009F440C08091B4
:101F8000E80083FD3EC08091E80082FD30C0809172
:101F9000E80080FF1DC08091F200282F30E008C0CB
:101FA00084918093F1003196415050402F5F3F4F14
:101FB0004115510519F02031310590F390E02031A1
:101FC000310509F491E08091E8008E778093E80074
:101FD0004115510569F6992359F609C08EB3882336
:101FE00061F0853061F08091E80083FD0AC0809146
:101FF000E80082FFF3CF80E0089582E0089583E057
:10200000089581E00895EF92FF920F931F93CF936D
:10201000DF939C010091910110919201061717071F
:1020200018F4790190E03EC06115710511F08B0143
:10203000F8CF8091E8008E778093E80000E010E010
:10204000F0CF8EB3882309F442C0853009F441C033
:102050008091E80083FD3FC08091E80082FD31C09F
:102060008091E80080FF1EC08091F200C82FD0E070
:102070000AC0C7019ED38093F1000894E11CF11CB3
:102080000150104021960115110519F0C031D105FC
:1020900080F390E0609709F491E08091E8008E77FA
:1020A0008093E8000115110561F6992351F609C0E6
:1020B0008EB3882361F0853061F08091E80083FD64
:1020C0000AC08091E80082FFF3CF80E005C082E083
:1020D00003C083E001C081E0DF91CF911F910F9198
:1020E000FF90EF900895BF92CF92DF92EF92FF9210
:1020F0000F931F93CF93DF938C01EB016A011CD1E7
:10210000B82E8823B9F521970C0F1D1F2196C114F5
:10211000D10439F0F60180819181C81BD90B081BCD
:10212000190BEE24FF2424C08091E80085FD16C021
:102130008091E8008B778093E80027D3C114D10405
:1021400049F0F601808191818E0D9F1D91838083DE
:1021500085E011C0F1D0882359F00DC08091F100C5
:10216000F80180830150104021970894E11CF11C74
:102170002097D1F68B2DDF91CF911F910F91FF907A
:10218000EF90DF90CF90BF900895BF92CF92DF92F3
:10219000EF92FF920F931F93CF93DF93182F092F86
:1021A0007B016A01C9D0B82E8823B1F5812F902F09
:1021B0009C01E901C114D10439F0F60180819181BB
:1021C000E81AF90AC80FD91F00E010E022C0809178
:1021D000E80085FD16C08091E8008B778093E800C9
:1021E000D4D2C114D10449F0F60180819181800FCD
:1021F000911F9183808385E010C09ED0882349F091
:102200000CC08091F10089930894E108F1080F5FF8
:102210001F4FE114F104D9F68B2DDF91CF911F915F
:102220000F91FF90EF90DF90CF90BF900895BF92F5
:10223000CF92DF92EF92FF920F931F93CF93DF9392
:10224000182F092F7B016A0177D0B82E8823B1F5AA
:10225000812F902F9C01E901C114D10439F0F601BE
:1022600080819181E81AF90AC80FD91F00E010E0B7
:1022700022C08091E80085FD16C08091E8008E772D
:102280008093E80082D2C114D10449F0F601808124
:102290009181800F911F9183808385E010C04CD085
:1022A000882349F00CC089918093F1000894E108DB
:1022B000F1080F5F1F4FE114F104D9F68B2DDF9168
:1022C000CF911F910F91FF90EF90DF90CF90BF9033
:1022D00008958F708093E9008091EB008160809376
:1022E000EB001092ED006093EC004093ED008091C4
:1022F000EE00881F8827881F089580918B0188230E
:102300008CF403C08EB38823B1F08091E80082FF83
:10231000F9CF8091E8008B778093E80008958EB321
:10232000882349F08091E80080FFF9CF8091E80090
:102330008E778093E80008954091E4005091E50085
:1023400024E68091EC0080FF23C08091E80080FDAE
:102350001DC08EB3882311F482E00895853011F4F6
:1023600083E008958091EB0085FF02C081E008952D
:102370008091E4009091E5008417950711F32223E2
:1023800011F484E008952150AC01DBCF80E0089582
:102390008091E80082FFDDCFF9CF3CD03ED0809124
:1023A000D8008F778093D8008091D8008068809380
:1023B000D8008091D8008F7D8093D80084E089BDBB
:1023C00086E089BD09B400FEFDCF1EBA10928901D6
:1023D00080E060E042E17DDF8091E1008E7F8093CC
:1023E000E1008091E20081608093E2008091E20050
:1023F00088608093E2008091E0008E7F8093E0000F
:102400000895E3E6F0E080818E7F808381E0809311
:102410008A01C3CF1092E20008951092E10008955E
:102420001F920F920FB60F9211242F933F934F9349
:102430005F936F937F938F939F93AF93BF93EF932C
:10244000FF938091E10080FF17C08091E20080FF40
:1024500013C08091E2008E7F8093E2008091E200C1
:1024600080618093E2008091D80080628093D800E0
:1024700019BC1EBA0E941C018091E10084FF2FC08C
:102480008091E20084FF2BC084E089BD86E089BD95
:1024900009B400FEFDCF8091D8008F7D8093D800D5
:1024A0008091E1008F7E8093E1008091E2008F7E39
:1024B0008093E2008091E20081608093E20080914D
:1024C0008901882311F084E007C08091E30087FD33
:1024D00002C081E001C083E08EBB0E9417018091A1
:1024E000E10083FF21C08091E20083FF1DC0809145
:1024F000E100877F8093E10082E08EBB109289012A
:102500008091E1008E7F8093E1008091E2008E7FD8
:102510008093E2008091E20080618093E20080E09D
:1025200060E042E1D6DE30D1FF91EF91BF91AF91F3
:102530009F918F917F916F915F914F913F912F91DB
:102540000F900FBE0F901F9018951F93DF93CF939E
:1025500000D00F92CDB7DEB7EBE8F1E08091F1004B
:10256000819381E0E339F807C9F70ED18091E80043
:1025700083FFF5C080918B0190918C01953009F417
:102580006FC0963040F4913091F1913070F09330FB
:1025900009F0E5C02CC0983009F4B3C0993009F4B3
:1025A000C2C0963009F0DBC07DC0803811F490E0E5
:1025B00014C0823809F0D3C080918F018F7080934E
:1025C000E9008091EB0090E025E0969587952A95AB
:1025D000E1F7982F91701092E9008091E800877FD1
:1025E0008093E8009093F1001092F10095C0882349
:1025F00019F0823009F0B3C08F71823009F0AFC09A
:1026000080918D01882331F520918F012F7009F47D
:10261000A6C02093E9008091EB0080FF1BC093309F
:1026200021F48091EB00806213C08091EB00806107
:102630008093EB0081E090E002C0880F991F2A95FB
:10264000E2F78093EA001092EA008091EB00886044
:102650008093EB001092E9008091E800877F5FC0D3
:10266000882309F07CC010918D011F778091E300D1
:102670008078812B8093E3008091E800877F8093AE
:10268000E8003BDE8091E80080FFFCCF8091E30012
:1026900080688093E300112311F482E001C083E09D
:1026A0008EBB5DC08058823008F059C080918D018A
:1026B00090918E0160918F01AE014E5F5F4F9E0140
:1026C0002F5F3F4F0E942101BC01009709F447C0D2
:1026D0008091E800877F8093E8002981222321F4FC
:1026E0008A819B812DDC07C08A819B81213011F476
:1026F0008ADC01C0C3DB8091E8008B778093E8001F
:102700002EC0803861F58091E800877F8093E800D3
:10271000809189018093F1008091E8008E77809309
:10272000E800EBDD1CC08823D1F490918D0192303C
:10273000B0F48091E800877F8093E800909389014E
:10274000DCDD80918901882331F48091E30087FDED
:1027500002C081E001C084E08EBB0E9438018091FC
:10276000E80083FF0AC08091E800877F8093E8003B
:102770008091EB0080628093EB000F900F900F90A0
:10278000CF91DF911F91089508951F938EB38823F1
:1027900071F01091E9008091EC001092E9008091B5
:1027A000E80083FF01C0D1DE1F701093E9001F9184
:1027B0000895F999FECF92BD81BDF89A992780B509
:1027C0000895262FF999FECF92BD81BDF89A019701
:1027D00000B4021639F01FBA20BD0FB6F894FA9A69
:0A27E000F99A0FBE0895F894FFCF98
:1027EA0009022000010100C0320904000002FF00B2
:1027FA0000000705820240000A0705020240000A9B
:10280A001C0330003000300032003000300030004D
:10281A003100320033003400350000000000415618
:10282A00524953505F4D4B320080010081010090A4
:10283A0001009101019201189401219803069E0357
:10284A0001A10100A4030001C001000120003332EC
:10285A001289AB45CDD888FF1289AB45CDD888FF00
:00000001FF
